:10000000831602309F0089018601BF3087002430AB
:100010009800813099008312903098000730890051
:100020008317A03084000430A600FF3086006C20C7
:10003000003086008C1E1A2818194D28981855284B
:100040001A088000840AA60B1A2800308000A0300D
:1000500084000530A6000008A50026084620A70059
:10006000A50C031C42284428091100000915A70B00
:100070003028840AA60B2B288914000009100000E0
:1000800009141028891034288914342882070000A4
:10009000023408340834083407340F3086006C20EA
:1000A000003086001A08981C1028F03086006C205A
:1000B00000308600181218161028A530A000000085
:1000C0000000A00B612808006330A10000000000C0
:1000D0005D20A10B682808006330A2006230A300F5
:1000E0000330A40000006420A20B73285D20A30B42
:0800F0007628A40B7928080012
:00000001FF
